:100000000C9417060C943C290C9469290C943F0617
:100010000C943F060C943F060C943F060C943F064C
:100020000C943F060C943F060C94C00C0C943F06B5
:100030000C943F060C943F060C943F060C943F062C
:100040000C9496290C943F060C94502D0C948B2DF7
:100050000C943F060C943F060C943F060C943F060C
:100060000C943F060C943F06901C971C971C901C08
:10007000971C971C971C971C971C971C971C971CE8
:10008000971C971C971C971C971C051C971C971C6A
:10009000971C971C971C681B971C971C971C971CF8
:1000A000971C971C971C971C971C971C971C971CB8
:1000B000971C971C971C111C111C111C111C111C46
:1000C000111C111C111C111C971C971C971C971CB0
:1000D000971C971C6D1B101C101C101C101C971CCF
:1000E000211C291C311C391C411C491C511C591C48
:1000F000631C6D1C771C811CB41B741B971C971C04
:10010000971C971C051C971C971C971C971C971CE9
:10011000971C971C971C0F1C0F1C0F1C0F1C971C67
:10012000211C291C311C391C411C491C511C591C07
:10013000631C6D1C771C811CB41B741B971C971CC3
:10014000971C971C051CC81CC81CC81CC81CC81CB4
:10015000C81CC81CC81CC81CC81CC81CC81CC81C7F
:10016000E81DE81DE81DE81DE81DE81D0F1D191D0F
:10017000231D2D1D931D9D1DAB1DBC1D591EC91E8C
:100180009A1E9F1EA41EA91EAE1EB31EB81EC91E17
:10019000C31ECF25E425F025F92506262C26342676
:1001A00057264426456E746572206D656E752E2E39
:1001B0002E00546F67676C6564206D6963726F50C1
:1001C000504D00546F67676C656420696E76657288
:1001D0007465642050504D2100546F67676C6564EE
:1001E000205458206D7574696E672100546F6767DD
:1001F0006C65642074656C656D657472792100505E
:10020000726F746F636F6C206572726F72207769A2
:1002100074682052580054696D656F757420776852
:10022000656E20636F6E6E656374696E6720746FB0
:1002300020525800507265737320616E79206B658F
:100240007920746F2063616E63656C00436F6E6E1E
:10025000656374696E6720746F2052582C20706F2C
:100260007765722075702074686520525820287751
:100270006974682062696E6420706C7567206966B5
:10028000206E6F74207573696E6720616C77617979
:10029000732062696E642900546F67676C6564201F
:1002A00027696D6D656469617465206F757470751B
:1002B000742700546F67676C65642027736C6176E0
:1002C00065206D6F64652700546F67676C656420F7
:1002D00027616C776179732062696E642700546FBF
:1002E00067676C65642050504D206368616E6E6571
:1002F0006C206C696D6974005365742052535349C6
:1003000020696E6A656374696F6E206368616E6EE2
:10031000656C2028303D3D64697361626C6529001D
:100320005365742050504D206D696E696D756D2058
:1003300073796E630053657420626561636F6E202C
:10034000696E74657276616C0053657420626561D4
:10035000636F6E2064656C6179005365742062651B
:1003600061636F6E206672657175656E6379206971
:100370006E20487A3A20303D64697361626C652C66
:100380002050783D504D52206368616E6E656C2040
:10039000782C2046783D465253206368616E6E6526
:1003A0006C2078005365742050574D2073746F7023
:1003B0002064656C61792028302064697361626C07
:1003C00065642C20312D323535203D3D20302E31D5
:1003D00073202D2035306D696E29005365742050CF
:1003E000504D2073746F702064656C6179202830E3
:1003F0002064697361626C65642C20312D3235355F
:10040000203D3D20302E3173202D2035306D696E1A
:100410002900536574206661696C736166652064A8
:10042000656C61792028302064697361626C656451
:100430002C20312D323535203D3D20302E3173209A
:100440002D2035306D696E29002A2A2A2A2A2A2A67
:100450002A2A2A2A2A2A2A2A2A2A2A2A2A2A2A2AFC
:100460002A2A2A2A2A2A0052582041636B656420CE
:100470002D2072657665727420737563636573737E
:1004800066756C21002A2A2A2A2A2A2A2A2A2A2A36
:100490002A2A2A2A2A2A2A2A2A2A2A2A2A2A2A2ABC
:1004A0002A2A002A2A2A2A2A2A2A2A2A2A2A2A2AD6
:1004B0002A2A2A2A2A2A2A2A2A2A2A2A2A2A2A2A9C
:1004C0000052582041636B6564202D207570646173
:1004D0007465207375636365737366756C21002A98
:1004E0002A2A2A2A2A2A2A2A2A2A2A2A2A2A2A2A6C
:1004F0002A2A2A2A2A2A2A2A2A2A2A2A0056616CE1
:1005000069642063686F69636573206172653A206E
:100510005B315D2D5B31365D20286368616E6E65F1
:100520006C20312D31362900536574206F7574703D
:10053000757420666F7220706F727420005B585D56
:100540002061626F7274206368616E6765732061F9
:100550006E64206578697420525820636F6E6669F6
:1005600067005B535D207361766520736574746901
:100570006E677320746F205258005B525D20726565
:10058000766572742052582073657474696E67734F
:1005900020746F2064656661756C747300557365B3
:1005A000206E756D62657273205B312D445D207421
:1005B0006F206564697420706F727473205B452DC1
:1005C000515D20666F722073657474696E67730085
:1005D000202D20726563656976657220636F6E6693
:1005E0006967757261746F722C207278207377203E
:1005F000000A0A6F70656E4C52536E672000536597
:10060000742073657269616C2062617564726174D3
:10061000653A200056616C69642063686F696365A0
:10062000733A2031202D20342B34202F2032202DDE
:100630002038202F2033202D20382B34202F203419
:10064000202D203132202F2035202D2031322B3407
:10065000202F2036202D203136005365742043682A
:10066000616E6E656C20636F6E6669673A20005339
:1006700065742044617461726174652028302D3284
:10068000293A200053657420486F70206368616EBA
:100690006E656C7320286D61782032342C20736570
:1006A0007061726174656420627920636F6D6D6141
:1006B00073292076616C69642076616C756573209E
:1006C000312D3235353A2000536574206368616EF0
:1006D0006E656C2073706163696E672028783130B5
:1006E0006B487A293A200053657420524620706F77
:1006F0007765722028302D37293A20005365742001
:100700005246206D616769632028686578292065F5
:100710002E672E20307844454144463030443A20FC
:10072000005365742062617365206672657175653A
:100730006E63792028696E20487A293A20005B5A36
:100740005D20656E74657220726563656976657299
:1007500020636F6E66696775726174696F6E20756C
:1007600074696C79005B465D20646973706C6179B3
:100770002061637475616C206672657175656E6366
:100780006965732075736564005B525D2063616CFD
:1007900063756C6174652072616E646F6D206B654A
:1007A0007920616E6420686F70206C697374005BDF
:1007B000495D207265696E697469616C697A65204A
:1007C00073657474696E677320746F20736B6574DE
:1007D00063682064656661756C7473005B585D20A6
:1007E000726576657274206368616E6765732061F7
:1007F0006E642065786974206D656E75005B535D6D
:1008000020736176652073657474696E67732074F4
:100810006F20454550524F4D20616E6420657869C8
:1008200074206D656E7500557365206E756D62651B
:100830007273205B302D395D20746F20656469749C
:1008400020706172616D657465727300202D205394
:10085000797374656D20636F6E6669677572617414
:10086000696F6E000A0A6F70656E4C52536E672096
:10087000005129204F7574707574206265666F721F
:1008800065206C696E6B20283D465329203A200074
:10089000502920536C617665206D6F646520286552
:1008A00078706572696D656E74616C293A20004FCD
:1008B000292054696D65642042494E4420617420AA
:1008C0007374617274757020203A20004E29205094
:1008D000504D206F7574707574206C696D69746506
:1008E0006420202020203A200044495341424C45B6
:1008F00044004D292050504D205253534920746FCD
:10090000206368616E6E656C202020203A20004CC8
:10091000292050504D206D696E696D756D20737979
:100920006E63202875732920203A200044495341E2
:10093000424C4544004B29204661696C73616665F1
:1009400020626561636F6E20696E74762E20283197
:100950002D32353573293A20004A29204661696CC9
:100960007361666520626561636F6E2064656C61AA
:10097000792028302D323535203D3E20313073200E
:100980002D203135306D696E293A200049292046E5
:1009900061696C7361666520626561636F6E206674
:1009A00072712E203A200048292050574D20737430
:1009B0006F702064656C6179202020202020203A0F
:1009C000200047292050504D2073746F70206465BB
:1009D0006C6179202020202020203A200046292008
:1009E0004661696C736166652064656C617920207D
:1009F00020202020203A200050574D206368616E4F
:100A00006E656C200066756E6374696F6E3A2000C7
:100A10002920706F72742000506F776572546F7761
:100A2000657200445446205548462033322D626991
:100A3000742031306368004F70656E4C52536E679E
:100A40005258206D696E6920342F36636800466CF9
:100A50007974726F6E2F4F72616E676552582055B0
:100A600048462038636800525820747970653A20EF
:100A70000044697361626C656400487A00203D3D02
:100A8000200043616C63756C617465642070616300
:100A90006B657420696E74657276616C3A200042F1
:100AA00029204D6963726F202868616C6629205087
:100AB000504D202020203A00412920496E76657251
:100AC0007465642050504D20696E20202020203A0B
:100AD000003029204D7574652062757A7A65722020
:100AE000286D6F73746C79293A0039292053657227
:100AF00069616C2062617564726174653A00736D3E
:100B0000617274506F7274004672536B7900547244
:100B1000616E73706172656E740044697361626CBA
:100B200065640038292054656C656D657472793A86
:100B300020202020202020003729204368616E6E6D
:100B4000656C20636F6E6669673A20200036292045
:100B500044617461726174652028302D32293A2015
:100B6000202000352920486F70206368616E6E6513
:100B70006C733A2020202020003429204368616EC5
:100B80006E656C2073706163696E673A2020003374
:100B90002920524620706F7765722028302D372922
:100BA0003A202020003229205246206D6167696377
:100BB0003A202020202020202020003129204261BE
:100BC0007365206672657175656E63793A202020C1
:100BD0000000000000240027002A0000000000257B
:100BE0000028002B0000000000230026002900043C
:100BF00004040404040404020202020202030303C4
:100C000003030301020408102040800102040810BD
:100C1000200102040810200000000700020100006B
:100C2000030406000000000000000000332F112420
:100C30001FBECFEFD8E0DEBFCDBF13E0A0E0B1E034
:100C4000E8EAF0E602C005900D92A839B107D9F79D
:100C500016E0A8E9B3E001C01D92AB35B107E1F79A
:100C60001CE0CEE2DCE004C02297FE010E942F309F
:100C7000CC32D107C9F70E94782F0C9452300C94D3
:100C80000000A0E0B0E0E7E4F6E00C94FE2FEC01F9
:100C9000A880B980CA80DB80A114B104C104D1044A
:100CA00041F484E2A82E89EDB82E8BE5C82E87E0AA
:100CB000D82EC601B5012DE133EF41E050E00E948E
:100CC000DB2F27EA31E440E050E00E94872F7B01D0
:100CD0008C01C601B5012DE133EF41E050E00E94E7
:100CE000DB2FCA01B9012CEE34EF4FEF5FEF0E940A
:100CF000872F6E0D7F1D801F911F97FF04C06150CD
:100D0000704080409048688379838A839B839B01ED
:100D1000AC015F77B901CA01CDB7DEB7EAE00C9448
:100D20001A300E944106089581EB92E00E9441062C
:100D300008956093B1027093B2028093B3029093CE
:100D4000B4020895A0E0B0E0E8EAF6E00C94F72FD2
:100D5000EC012B016A016115710519F0FB0191830A
:100D60008083C114D10449F0C6010297839728F00B
:100D700020E030E040E050E0DCC0A9908A2D90E017
:100D80000E944730892BC9F7FDE2AF1621F4A990E4
:100D90003324339405C08BE2A81609F4A9903324B8
:100DA000C114D10421F0E0E1CE16D10411F5F0E335
:100DB000AF1669F48881883711F0883541F4A9802D
:100DC000229682E0382A20E1C22ED12C12C0C11412
:100DD000D10479F4E0E3AE1659F199E9E92E99E9E5
:100DE000F92E99E9092F99E1192F8AE0C82ED12C03
:100DF0003AC0FAE0CF16D10491F080E1C816D104D0
:100E000029F0E8E0CE16D104F9F415C0BFEFEB2EBF
:100E1000BFEFFB2EBFEF0B2FBFE01B2F24C0A9E9B4
:100E2000EA2EA9E9FA2EA9E90A2FA9E11A2F1BC077
:100E3000F8E0CF2ED12CEFEFEE2EEFEFFE2EEFEFFE
:100E40000E2FEFE11E2F0FC09601442737FD40956E
:100E5000542F6FEF7FEF8FEF9FEF0E94B92FC901E3
:100E6000DA017C018D0120E030E040E050E060E0FC
:100E70003601882477FC8094982C70EDB72EBA0C3C
:100E8000F9E0FB1570F48A2D81548A3118F499EC3D
:100E9000B92E06C08A2D81568A3148F589EAB82EC6
:100EA000BA0C8B2D90E08C159D050CF56F3FE9F089
:100EB000E216F30604071507B8F0CA01B901A40148
:100EC00093010E94872F9B01AC018B2D90E0A0E045
:100ED000B0E0280F391F4A1F5B1F281739074A0740
:100EE0005B0710F061E001C06FEFA990C6CF41141D
:100EF000510451F0662311F0219703C031FE04C064
:100F00002297F201D183C08330FE07C050954095EF
:100F1000309521953F4F4F4F5F4F67FF0AC082E2E8
:100F200090E090935A06809359062FEF3FEF4FEFD2
:100F30005FEFB901CA01CDB7DEB7E1E10C94133020
:100F4000FC0188279927E89421912032E9F3293080
:100F500010F02E30C8F32B3241F02D3239F4689462
:100F600004C00E94F507820F911D219120532A3061
:100F7000C0F31EF4909581959F4F089548E953E082
:100F80000E94C3070895009731F4DA018D919C9176
:100F9000009709F40EC0DC01FB013D912191222351
:100FA00019F03217C9F3FACF332331F4DA011D9265
:100FB0001C928827992708951197AF93BF93FB013F
:100FC0003D912191321771F4332321F48827992719
:100FD000119702C01E921196FA01A193B0839F91BE
:100FE0008F910895222369F7EACF7AE0979F902D99
:100FF000879F802D910D1124089580919A0381304F
:1010000019F482E080939A0380919A03833019F453
:1010100084E080939A030895E3E0F0E089E0809310
:101020005700849190E08670863009F491E0892F12
:1010300008951F93182F0E940C08882379F09FB7FA
:1010400081E08093A105F894A89588E180936000E1
:1010500010936000112309F0A8959FBF1F91089578
:10106000382F20E080913305909134058227932713
:1010700040E061E270E19C01220F331F97FF04C042
:10108000C9018627972701C0C9014F5F483099F7EA
:101090009093340580933305089587E38093D003BC
:1010A00080E092ECA1E0B0E08093D1039093D20372
:1010B000A093D303B093D40387E08093DD0380E053
:1010C00091EAACEBB3E38093D5039093D603A0935E
:1010D000D703B093D80385E08093DE038DEE9EEFB7
:1010E000ADEABEED8093D9039093DA03A093DB03BE
:1010F000B093DC03AFEDB3E080E090E0863010F019
:10110000E0E004C0FC01EF57FC4FE081ED93019655
:101110008831910599F782E08093F7038AE0809304
:10112000F803089580E09EECADEEB4E380939D0358
:1011300090939E03A0939F03B093A00380E090E060
:10114000A0E0B0E58093A1039093A203A093A30332
:10115000B093A403E5EAF3E080E081938F5F8031F0
:10116000E1F708958436910520F4BC0180E090E019
:1011700025C08E3B910550F48A559040BC0180E01B
:1011800090E02AE030E040E050E016C0823D91055A
:1011900050F4845B9040BC0180E090E024E630E0B5
:1011A00040E050E009C08D5C9040BC0180E090E0E0
:1011B00028E532E040E050E00E94872F24E630E04E
:1011C00040E050E00E94872F089590E08C599F4F97
:1011D0000E94B2080895DC019896EC91F0E0E77067
:1011E000F070E758FC4F808108958F929F92AF92E4
:1011F000BF92CF92DF92EF92FF920F931F938C01D9
:101200000E94EB08D80197962C9130E043E150E022
:10121000249FF001259FF00D349FF00D1124EB5415
:10122000FD4F80809180A280B38090E00F96AA2726
:1012300097FDA095BA2FBC01CD0120E43FE14DE719
:1012400050E00E94872FA50194010E94B92F6901E7
:101250007A0180ED97E0A0E0B0E0C80ED91EEA1E4A
:10126000FB1ED80198968C91887181F060E07EEE2B
:101270008AEB9BE0A50194010E94B92F28513C4FB5
:101280004F4F5F4FC20ED31EE41EF51E87EE93E054
:10129000A0E0B0E0C80ED91EEA1EFB1EC701B601D1
:1012A00028EE33E040E050E00E94B92FCA01B901B6
:1012B00028EE33E040E050E00E94872F1F910F910D
:1012C000FF90EF90DF90CF90BF90AF909F908F9066
:1012D00008958F3F910509F010F480E0089522E011
:1012E0008030920710F481E008958050934010F010
:1012F00083E0089582E00895CF92DF92FF920F93EA
:101300001F93CF93DF93F82FEB016A01182F1695E7
:10131000E0E088819981D6018C938A819B81119626
:101320008C9311978C819D8112968C9312978E814C
:101330009F8113968C931397288139814A815B8111
:101340006C817D818E819F819295990F990F907C00
:10135000832F8370982B852F8370880F880F982B8D
:10136000872F83708295807F982B14969C9385E0BD
:1013700090E0C80ED91E2896EF5F1E1750F6F0FFBA
:1013800021C0888199810E946909F82E8A819B81F8
:101390000E946909182F8C819D810E946909082F7C
:1013A0008E819F810E946909F294FF0CFF0C70EC02
:1013B000F7221295107F1F29182B000F000F012B09
:1013C000D6010C93DF91CF911F910F91FF90DF9089
:1013D000CF90089523E08032920718F420E030E0A7
:1013E00026C023E0883E920748F49C012F513340E9
:1013F00054E0369527955A95E1F719C027E0803DCE
:10140000920720F49C012C5D334011C028E08839FC
:10141000920718F02FEF33E00AC09C01285C374098
:1014200044E0369527954A95E1F72D503C4FC90188
:1014300008958C30910548F49C0174E0220F331F0D
:101440007A95E1F7285D3C4F17C023E0843F92076F
:1014500020F49C0124523C4F0FC024E080309207BE
:1014600018F020E938E008C09C012657334F64E0AB
:10147000220F331F6A95E1F7C90108959C01369543
:10148000279525753575821B930B9C0136952795FD
:10149000369527952373337383739373280F391FFE
:1014A000C901E4E096958795EA95E1F7820F931FCD
:1014B0008F709F7021E031E0AC01429FC001439FDB
:1014C000900D529F900D1124892F0895882339F093
:1014D0002D9800002B9A00002D9A000008952D9859
:1014E00000002B9800002D9A000008952D9A00000E
:1014F00083B12D98000090E0B4E096958795BA9559
:10150000E1F7817008950F931F93082F5C9A2D982F
:101510005C9810E0802F80780E94660A000F1F5FA1
:101520001830C1F72D981F910F9108958F770E9461
:10153000830A08950F931F93082F10E0802F80785F
:101540000E94660A000F1F5F1830C1F72D981F9187
:101550000F9108950F931F932D9880E000E0182FAE
:10156000110F0E94760A810F0F5F0830C1F71F919B
:101570000F9108950E94960A0E94AA0A5C9A089503
:101580001F93162F80680E94830A812F0E949A0A57
:101590005C9A1F9108951F931091D9031827E0EDCD
:1015A000F3E0E80FF11D89E767850E94C00A8DE32B
:1015B000612F0E94C00A82E4612F0E94C00A1F911D
:1015C000089586E20E94BA0A08950F931F938C0132
:1015D0008CE1F80164810E94C00A8DE1F801658107
:1015E0000E94C00A8EE1F80166810E94C00A80E272
:1015F000F80167810E94C00A81E2F80160850E94BB
:10160000C00A82E2F80161850E94C00A83E2F80103
:1016100062850E94C00A84E2F80163850E94C00AC4
:1016200085E2F80164850E94C00A8AE2F8016585B6
:101630000E94C00A8EE6F80166850E94C00A8FE605
:10164000F80167850E94C00A80E7F80160890E945E
:10165000C00A81E7F80161890E94C00A82E7F801A7
:1016600062890E94C00A1F910F910895EF92FF9224
:101670000F931F93CF93DF937B018C01603028E39E
:1016800072072CE982072CE1920728F520E836E959
:1016900048E950E00E94B92FE9016897B90180E05C
:1016A00090E020E839E647E65FEF0E94872F6E0D55
:1016B0007F1D801F911F32E0660F771F881F991FC3
:1016C0003A95D1F721E732E040E050E00E94B92F8F
:1016D000890180E421C020E03DE241E351E00E9425
:1016E000B92FE9016897B90180E090E020E033ED7F
:1016F0004EEC5EEF0E94872F6E0D7F1D801F911FA5
:10170000660F771F881F991F21E732E040E050E005
:101710000E94B92F890180E69E012F71622F680F08
:1017200085E70E94C00A86E7612F0E94C00A87E70A
:10173000602F0E94C00ACDB7DEB7E6E00C941E30E1
:101740009F92AF92BF92CF92DF920F93DF93CF938E
:1017500000D000D0CDB7DEB7982E83E00E94BA0A41
:101760008093F90384E00E94BA0A8093FA0386E02A
:1017700060E00E94C00A87E061E00E94C00A89E040
:101780006FE70E94C00A8AE065E00E94C00A8BE011
:1017900062E10E94C00A8CE065E10E94C00A8DE00F
:1017A0006DEF0E94C00A8EE060E00E94C00A99209E
:1017B00019F084E193E008C08091F70323E1829F50
:1017C000C00111248B549D4F0E94E50A80E36CE810
:1017D0000E94C00A82E36FE00E94C00A83E362E4D1
:1017E0000E94C00A84E36AE00E94C00A85E36AE2BC
:1017F0000E94C00A86E36DE20E94C00A87E364ED9E
:101800000E94C00A88E360E00E94C00A89E360E0A9
:101810000E94C00A992049F065E8A62E61ECB62E18
:1018200061ECC62E6EEDD62E08C0A090D903B09004
:10183000DA03C090DB03D090DC030AE38D2D9927F7
:10184000AA27BB2789839A83AB83BC83802F6981B6
:101850000E94C00A802F8B5F69810E94C00ADC2C25
:10186000CB2CBA2CAA240F5F0E3341F783E46FEF21
:101870000E94C00A84E46FEF0E94C00A85E46FEF03
:101880000E94C00A86E46FEF0E94C00A992019F0F6
:101890008DE666E003C08DE66091DD030E94C00A1C
:1018A00089E760E00E94C00A8AE76091DE030E9437
:1018B000C00A83E760E00E94C00A84E760E00E94FB
:1018C000C00A992029F060E071EA8CEB93E308C02C
:1018D0006091D5037091D6038091D7039091D8037E
:1018E0000E94360B0F900F900F900F90CF91DF91C9
:1018F0000F91DF90CF90BF90AF909F90089587E0B9
:1019000061E00E94C00A8EE764E20E94C00A88E09B
:1019100063E00E94C00A88E060E00E94C00A87E09D
:1019200065E00E94C00A85E062E00E94C00A83E090
:101930000E94BA0A8093F90384E00E94BA0A809355
:10194000FA030895582F40919E04842F90E0FC01E3
:10195000EF70F0709F012F5F3F4F74E09595879572
:101960007A95E1F72817390751F0E257FB4F50837A
:10197000842F8F5F8F70407F842B80939E04089507
:101980001F920F920FB60F9211241F932F933F9324
:101990004F935F936F937F938F939F93AF93BF9377
:1019A000CF93DF93EF93FF93C0918600D091870090
:1019B0002091E0043091E1048091BF04882309F074
:1019C00062C0BE01621B730B2091A1033091A20380
:1019D0004091A3035091A40325FD02C0769567951D
:1019E00089E0653C7807B8F1809147031CE1569582
:1019F0004795379527951A95D1F72115310541055A
:101A0000510521F421E030E040E050E090E0A0E01A
:101A1000B0E0281739074A075B07D0F480914703E5
:101A20008F3FB1F020E00EC0E22FF0E0EE0FFF1F7D
:101A3000DF01A054BB4F8D919C91E95DFC4F9183D8
:101A400080832F5F80914703281770F31092BE04A4
:101A50001092470318C082E06D3B780760F18091D7
:101A60004703803140F510914703CB010E94EA09FA
:101A7000E12FF0E0EE0FFF1FE054FB4F91838083D6
:101A80001F5F10934703D093E104C093E004FF91DC
:101A9000EF91DF91CF91BF91AF919F918F917F9106
:101AA0006F915F914F913F912F911F910F900FBEBA
:101AB0000F901F9018958FEF80934703E4CF83E03A
:101AC000809380008AE9809381008091A10386FD44
:101AD00005C0809181008064809381008FEF9FEF2B
:101AE000909389008093880080916F00806280933A
:101AF0006F0008956F3018F086958058089589E03A
:101B0000689F802D11240895882319F460E071E006
:101B100002C063E071E087E396E00E943B2D0895E8
:101B2000A0E0B0E0E6E9FDE00C940030182F0E9440
:101B3000EC299B01AC0180912D0590912E05A0917F
:101B40002F05B091300569017A01C81AD90AEA0A4D
:101B5000FB0AD701C60189589341A040B04010F05C
:101B600010922C0520932D0530932E0540932F05C0
:101B7000509330052091BF04822F81508230E8F5C8
:101B800080912C05882309F44FC1813011F482E043
:101B9000BCC1803108F035C1E82FF0E0E054FB4FC4
:101BA00010838F5F80932C05803109F0B0C1A2ECC7
:101BB000B4E0213039F41196EC911197E695E69551
:101BC0008C9109C08D919C911197E92FE695E6952E
:101BD000E69596958795E03140F4F0E090E0EE0FC1
:101BE000FF1FE95DFC4F918380831092BE04129623
:101BF00084E0A03DB807E9F68AC1233009F004C1AA
:101C000080912C05882321F41F3009F080C10CC17C
:101C1000883130F4E82FF0E0E154FB4F108374C1B9
:101C2000883109F0EEC0112309F0EBC0C0E0D0E02C
:101C30000BE010E0DE0163E0AA0FBB1F6A95E1F73D
:101C4000C09FB001C19F700DD09F700D1124FB018A
:101C5000E054FB4F80812181922F97709595879555
:101C6000FD01EE0FFF1FE95DFC4F91838083FB01B7
:101C7000EF53FB4F30813695369536952181422FB3
:101C80004295440F407E842F832B269526952695DA
:101C9000922F977095958795FD01EE0FFF1FE75DD9
:101CA000FC4F91838083FB01EE53FB4F8081829533
:101CB0008695869583704181942F990F990F292FCE
:101CC000282B429546954695437082818170880FF6
:101CD000880F382F342B35952795FD01EE0FFF1F08
:101CE000E55DFC4F31832083FB01EC53FB4F3081DA
:101CF00036952181422F479544274795842F832B82
:101D00002695922F977095958795FD01EE0FFF1FF1
:101D1000E35DFC4F91838083FB01EB53FB4F3081EC
:101D200032953F702181422F4295407F842F832B33
:101D300022952F70922F977095958795FD01EE0F44
:101D4000FF1FE15DFC4F91838083FB01EA53FB4F52
:101D50008081881F8827881F4181942F990F292F00
:101D6000282B441F4427441F82818370880F382FFB
:101D7000342B35952795FD01EE0FFF1FEF5CFC4FCF
:101D800031832083FB01E853FB4F30813695369534
:101D90002181422F4295440F440F407C842F832B96
:101DA00026952695922F977095958795AA0FBB1F1C
:101DB000FD01ED5CFC4F9183808367537B4FFB01FA
:101DC00020812295269527704181342F330F330FC0
:101DD000330F832F822B942F92959695977095951C
:101DE0008795AB5CBC4F11969C938E932196C23025
:101DF000D10509F01FCF8091D60483FD02C0109257
:101E0000BE0410922C0583C0243009F080C040919C
:101E10002C05442359F4183AB1F410923405109269
:101E2000330588EA0E94300881E06FC0413019F420
:101E30001093310504C0423031F410933205812FE4
:101E40000E9430085DC060913205262F30E0220FDD
:101E5000331FE42FF0E0C90102968E179F0734F07C
:101E6000433268F7E354FB4F1083E9CF2D5F3F4FB8
:101E70004091330550913405E217F30749F4912F4F
:101E800080E048275927509334054093330538C0E4
:101E9000812F90E04817590789F5809131058130ED
:101EA00069F5613118F080E180933205D0903205F8
:101EB00040ECE42E44E0F42E00E010E01BC0F701FB
:101EC000D081C0E0818190E08C2B9D2B33E09695F2
:101ED00087953A95E1F70E94EA09F801EE0FFF1F96
:101EE000E95DFC4F918380830F5F1F4F82E090E09C
:101EF000E80EF91E0D1518F31092BE0410922C0571
:101F000080912C05882319F08F5F80932C05CDB725
:101F1000DEB7E8E00C941C30FF920F931F93CF9331
:101F2000DF93182F092FF62E8EE30E94C00A212F6F
:101F3000302FC901EC0110E005C08FE769910E94C4
:101F4000C00A1F5F1F15C8F385E064E00E94C00A45
:101F500083E00E94BA0A8093F90384E00E94BA0ADF
:101F60008093FA030E94EC296093FB037093FC03B7
:101F70008093FD039093FE0387E069E00E94C00A0E
:101F800081E080939A03CDB7DEB7E5E00C941F3073
:101F90000E948C0F80919A038130D9F40E94EC2921
:101FA0002091FB033091FC034091FD035091FE030F
:101FB000621B730B840B950B605A764881409040EE
:101FC00040F4E8CF87E396E067E071E00E943B2DA4
:101FD000089580919A038130A9F3089587E396E0EC
:101FE0006EE70E94F32E0895A0E0B0E0EAEFFFE074
:101FF0000C94FF2F6C0187E396E06EE70E94F32EAE
:10200000760100E010E0C0E0D0E0B0E2BB2E0AC0F4
:102010000830110521F49E012095F60120870894CF
:10202000E11CF11CF7016081862F8D57823040F44E
:1020300087E396E06DE70E94F32EF70160816B2540
:1020400087E396E00E94F32E0115110551F0F70188
:1020500080819E01280F311DC32FDD27C20FD31FA2
:10206000D0700F5F1F4F0930110591F6CDB7DEB765
:10207000E9E00C941B30A9E0B0E0E1E4F0E10C945D
:102080000630382FE62F8091A30490E0019664E299
:1020900070E00E94A62F982F8093A30488E989837B
:1020A00080E18A83913071F0913028F0923099F07C
:1020B0009330E1F416C085E08B8381EF8C832F5F32
:1020C0002D8317C09B8381EF8C8384E6489FC001DA
:1020D00011249D830EC084E08B8381EF8C833D832C
:1020E00008C09B8381EF8C83ED8303C00E94EE0FB9
:1020F00004C0CE0101960E94F40F2996E2E00C94F0
:1021000022300F931F93CF93DF93182F092F87E36C
:1021100096E06EE70E94F32E212F302FC901EC01CB
:1021200010E000E288818D57823040F487E396E02A
:102130006DE70E94F32E88818027888387E396E0ED
:1021400069910E94F32E1F5F193061F787E396E0D3
:102150006EE70E94F32EDF91CF911F910F910895AA
:10216000A9E0B0E0E6EBF0E10C940630382F809166
:10217000A304882379F48EEF89833A836B83842FB9
:1021800090E0959587958C832D83198618861F82FC
:102190001E822FC040919E04842F90E09C012F70DE
:1021A000307054E0959587955A95E1F7821793071B
:1021B00021F18DEF89831A821B82DE01149620E0C3
:1021C00008C0E257FB4F80818D93405F2F5F263020
:1021D00069F0842F90E0FC0134E0F595E7953A959D
:1021E000E1F78F709070E817F90759F740939E0454
:1021F0002A83CE0101960E9481108091A30490E071
:10220000019666E070E00E94A62F8093A3042996B1
:10221000E2E00C9422309F92AF92BF92CF92DF9275
:10222000EF92FF920F931F93B82EA62ED42EC22E9C
:10223000902E0E94EC297B018C0180918D042091CD
:102240009F043091A0044091A1045091A2048823DE
:10225000B1F0D801C701821B930BA40BB50B815EB3
:102260009E42A040B04020F12C2DDC1408F42D2D0E
:102270008B2D6A2D422F292D0E943B1011C0D801B1
:10228000C701821B930BA40BB50B81539547A0404C
:10229000B04070F08B2D6A2D4D2D2C2D0E94B0106A
:1022A000E0929F04F092A0040093A1041093A20472
:1022B0001F910F91FF90EF90DF90CF90BF90AF9064
:1022C0009F90089587E396E0609100040E94F32EAA
:1022D00008951F93182F87E396E0612F0E94F32E35
:1022E000809100048127809300041F9108951F931B
:1022F000192F0E946911812F0E9469111F91089561
:10230000DF92EF92FF920F931F93D82E7B011092D2
:10231000000407E316E0C80165EB0E94F32EC80134
:1023200062E60E94F32E8D2D0E946911C7010E9462
:1023300077111F910F91FF90EF90DF900895E82F94
:10234000F0E0E456FC4FE185E03148F4F0E0EE0FB8
:10235000FF1FE95DFC4F0190F081E02D0DC0E031E1
:1023600029F0E13129F0E0E0F2E006C082E101C0AD
:1023700083E10E94402BFC01CF0108958CE060E0D6
:102380000E94712A8BE061E00E94712A8DE061E079
:102390000E94712A82E060E00E94712A84E061E07C
:1023A0000E94712A0895EF92FF920F931F93009756
:1023B00071F19C0140E050E068E478EE81E090E04B
:1023C0000E94DB2FC901DA017C018D0183E161E00C
:1023D0000E94DD2A8FEFE816F1040105110539F09E
:1023E00030F0FFEFEF2EF12C012D112D0AC0E1147A
:1023F000F1040105110529F4E1E0EE2EF12C012D87
:10240000112DE092B3008091B000806107C083E19C
:1024100060E00E94DD2A8091B0008F7E8093B00042
:102420001F910F91FF90EF900895A0E2B0E0EBE1D3
:10243000F2E10C94FE2F8CE00E94BA0A882389F501
:1024400087E396E063E171E00E943B2D5E9A409A3B
:1024500080E00E94A00B0E947F0C5E98409821C0F3
:1024600087E396E00E94BA2E482F8091BF0488230C
:1024700021F0842F0E94900D14C080912A05E82F2E
:10248000F0E031969F012F713070319780912905CE
:1024900090E02817390729F0E050FB4F4083209344
:1024A0002A0587E396E00E94802E892BC9F6809149
:1024B0009A03843009F08EC00E94EC296093AE0428
:1024C0007093AF048093B0049093B10461157105CB
:1024D0008105910561F481E090E0A0E0B0E0809397
:1024E000AE049093AF04A093B004B093B104809174
:1024F000BA049091BB0481609093BB048093BA04AA
:1025000083E080939A038FE70E94960A07EF14E016
:102510000E94AA0AF80181938F01F5E000301F079D
:10252000B9F74091E2048091F704282F30E0842F1E
:1025300090E08227932786FF40C080E4482740939D
:10254000E204C90188739070C89709F510E014C0BF
:102550001F5F8091F803E12FF0E084FF06C0E9508F
:10256000FB4F80810E94A20C07C0E950FB4F87E31C
:1025700096E060810E94F32E212F30E08091F704D5
:1025800090E0877090708217930714F716C02F732E
:102590003070232B91F48091F8048093B2048091E1
:1025A000F9048093B4048091FA048093B504809177
:1025B000FD048093BC041092BD0480912B058130F2
:1025C00019F482E080932B0580912B05833011F460
:1025D00010922B050E94EC295B016C018091B604DE
:1025E0009091B704A091B804B091B9040097A105E7
:1025F000B105C9F086017501E81AF90A0A0B1B0B2F
:10260000D801C701885B9B40A040B04060F00E94A9
:10261000E10A8093B3041092B6041092B7041092AA
:10262000B8041092B90480ED93E00E94F50820915F
:10263000AA043091AB044091AC045091AD048601E2
:102640007501E21AF30A040B150BE616F7060807E4
:10265000190708F411C1A092AA04B092AB04C09269
:10266000AC04D092AD04A8958091BE048830A0F04F
:102670008091A1039091A203A091A303B091A40320
:102680002CE1B695A795979587952A95D1F7009750
:10269000A105B10509F090C18091BE048F5F8093C0
:1026A000BE04E090AE04F090AF040091B00410912D
:1026B000B104E114F1040105110511F180ED93E07D
:1026C0000E94F508AE18BF08C00AD10A6A157B053A
:1026D0008C059D0588F48091A10384FD04C080EDE4
:1026E00097E00E94D3111092AE041092AF041092A2
:1026F000B0041092B10404C080E090E00E94D311B5
:102700009091E204907C9093E20400912A0510914C
:1027100029050117B1F180912B05823091F5905870
:102720009093E20480ED93E00E94EB08893010F072
:1027300048E002C0482F415030E013C03F5FA32F54
:10274000B0E0812F90E0FC01E050FB4F2081FD01C3
:10275000EE51FB4F2083A05EBA4F2C930196182FA9
:102760001F71341710F4101749F710932905832FA0
:10277000895C9091E204892B8093E20430932005D8
:102780001AC020912B052430D1F490912005E1E26C
:10279000F5E0A3EEB4E0292F30E02E0F3F1F02C07A
:1027A00081918D93E217F307D9F7995C8091E20448
:1027B000982B9093E20483E080932B0539C080919D
:1027C000A504823031F491609093E2045E9A409ABD
:1027D00010C09093E2045E984098222319F481E09F
:1027E00080932B0580912B05833019F484E080932E
:1027F0002B05F89405EA13E07E010894E11CF11C16
:10280000F80181918F010E949F11F70181939193AB
:102810007F01F3E0053B1F0799F78091F80387706C
:10282000BE016F5F7F4F43EE54E00E947C097894B5
:102830005D9A419A8091A4040E94CB0A80ED93E0B6
:102840000E94EB08682F82EE94E00E948C0FE091CA
:10285000A404EF5FE093A404E83131F0F0E0E0532A
:10286000FC4F8785882341F41092A40405C05E9A2A
:10287000409A89E08093BE048091F803887171F1D9
:1028800080919A03823051F58091BA049091BB04F3
:10289000880F991F9093BB048093BA0483E08093C0
:1028A0009A030E947F0C0E94EC296093B6047093F7
:1028B000B7048093B8049093B9046115710581053C
:1028C000910561F481E090E0A0E0B0E08093B6046F
:1028D0009093B704A093B804B093B9048091F8031F
:1028E00084FF1EC08091BA049091BB048E7F0E9429
:1028F0003E0A182F8091B2046091BC040E947A0DA8
:10290000082F8091B304612F0E947A0D282F8091A7
:10291000B4046091B504402F00919B030E940B11F9
:102920005D9841988091A5048130D1F0813020F0EC
:10293000823009F047C034C082E10E94102B892BFD
:1029400009F040C081E08093A5040E94DE296093D5
:10295000A6047093A7048093A8049093A90432C09E
:1029600082E10E94102B892B21F50E94DE29209103
:10297000A6043091A7044091A8045091A904621BB9
:10298000730B840B950B695E734080409040D0F0D0
:1029900082E08093A50480ED97E00E94D31112C0DD
:1029A00082E10E94102B892B69F080E090E00E9468
:1029B000D3111092A50406C08091BE04883009F09E
:1029C00058CF55CFA096EAE00C941A3083E161E02D
:1029D0000E94712A83E160E00E94DD2A82E08093F8
:1029E000B00085E08093B10083E061E00E94712A2D
:1029F00083E060E00E94DD2A08951F93182F0E9453
:102A0000EC2960939F047093A0048093A104909399
:102A1000A20410938D04112329F440E855E260E0EC
:102A200070E004C040E051EE60E070E087E396E0C3
:102A30000E94F92D1F910895ACE1B0E0E2E2F5E1CA
:102A40000C94FE2F0E94EC297B018C0181E00E94F6
:102A5000A00B54E7A52E6E010894C11CD11C43E0C5
:102A6000B42EA982C60161E00E94C80FB0929A03F9
:102A70000E947F0C6AEF70E080E090E00E94122AD2
:102A800080919A03833009F07DC087E396E00E942D
:102A9000802E892B09F076C00E94EC296E197F09DF
:102AA000800B910B6058734C894C914008F06AC0C0
:102AB000D8CF8FE70E94960A0E94AA0A843509F0AF
:102AC0005CC089830E94AA0A182F00E010938C042E
:102AD00000938B040E94AA0A080F111D10938C0406
:102AE00000938B040E94AA0A80938A040E94AA0A77
:102AF00080938904813108F040C0FF2407C00E9400
:102B0000AA0A07591B4FF8018083F3940F2D10E098
:102B10008091890490E0880F991F0817190778F3AE
:102B200080E78983CE01019661E00E94C80F83E0AF
:102B300080939A030E947F0C62E370E080E090E053
:102B40000E94122A80919A038330A9F08FE70E9495
:102B5000960A0E94AA0A803581F4898305EB13E066
:102B60000E94AA0AF80181938F01F3E0003D1F073C
:102B7000B9F781E003C082E001C083E06C96EAE02F
:102B80000C941A3080919A03833009F092CFF3CFDE
:102B900083E00E94BA0A8093F90384E00E94BA0A93
:102BA0008093FA0387E061E00E94C00A6AE070E067
:102BB00080E090E00E94122A0E947F0C000008959D
:102BC0000F931F93082F19C05E9A409A64E670E035
:102BD00080E090E00E94122A5E98409864E670E0DF
:102BE00080E090E00E94122A1F5F101768F36CE2E9
:102BF00071E080E090E00E94122A10E0F6CF482FAA
:102C0000392F25E00DC0F999FECF1FBA842F932FDD
:102C100092BD81BD60BD0FB6F894FA9AF99A0FBEC5
:102C2000215059F0F999FECF842F932F92BD81BD89
:102C3000F89A80B5681739F7089582E00E94E01588
:102C40000895A0E0B0E0E7E2F6E10C94F72F482EFB
:102C5000562EEE24FF2488249924C0E0D0E0CC2412
:102C6000DD2416E4312E04C055245394CC24DD24F5
:102C7000442069F480919B03839DE0011124BCE909
:102C8000EB2EB3E0FB2EA9E18A2E912C1DC021E092
:102C9000421671F480919B03839DE00111246B9691
:102CA000F0EDEF2EF3E0FF2EE9E28E2E912C0CC01A
:102CB00032E0431649F47BE9E72E73E0F72E61E03A
:102CC000862E912CC8E1D1E03E016C0C7D1C109247
:102CD000340510923305E3011BC0552059F4F999CE
:102CE000FECFD2BDC1BDF89A80B5F701E00FF11F4C
:102CF000808307C0F701E00FF11FCE0160810E94C1
:102D0000FF150E0D1F1DF80180810E9430082196CD
:102D10009E012619022F10E008151905F0F2CE01C8
:102D20005520D9F4F999FECFD2BDC1BDF89A20B58E
:102D3000F999FECF2196D2BDC1BD2197F89A80B5F1
:102D400090E0B22EAA248A299B2920913305309144
:102D500034052817390759F487CF21966091340537
:102D60000E94FF15CE01609133050E94FF1580E29D
:102D700091E0C80ED91E91EEC91692E0D90608F46A
:102D800077CF852DCDB7DEB7E1E10C94133080E02D
:102D900061E00E94211681E061E00E942116089501
:102DA00080E060E00E942116882331F081E060E03D
:102DB0000E942116882331F40E9492080E944D0837
:102DC0000E94C716089582E061E00E9421160895CE
:102DD00082E060E00E94211680919B03843020F005
:102DE00010929B030E94E31608951F93182F0E94D0
:102DF000E81680919B03811731F0143020F4109372
:102E00009B030E94E3161F9108951092670485E6C4
:102E1000E2E0F4E0DF011D928A95E9F708951F933F
:102E2000182F8F3711F08830E1F5E0916704EE2319
:102E300009F455C0E150E0936704F0E0EE5FFB4F0A
:102E4000108287E396E06DE00E94F32E10E00AC046
:102E5000E12FF0E0EE5FFB4F87E396E060810E9498
:102E6000F32E1F5F80916704181790F387E396E0B5
:102E700060E20E94F32E87E396E06DE00E94F32E5D
:102E800010E00AC0E12FF0E0EE5FFB4F87E396E031
:102E900060810E94F32E1F5F80916704181790F3E2
:102EA0001CC08B3119F40E9405171FC08D30E9F04A
:102EB0008A30D9F080916704843688F487E396E0FD
:102EC000612F0E94F32E80916704E82FF0E0EE5FFF
:102ED000FB4F10838F5F8093670480E007C087E318
:102EE00096E067E00E94A72BF8CF81E01F9108953C
:102EF0001F93CF93DF93CFEDD3E010E03BC087E388
:102F000096E062E271E00E94382D87E396E0612F3F
:102F10004AE050E00E94B52C87E396E06FE271E052
:102F20000E94382D699170E080E090E02091DE03EE
:102F300030E040E050E00E94872F20E137E240E09F
:102F400050E00E94872FDC01CB014091D5035091C6
:102F5000D6036091D7037091D803480F591F6A1F99
:102F60007B1F87E396E02AE030E00E947C2C1F5F05
:102F7000183119F08881882311F6DF91CF911F91C4
:102F80000895EF92FF920F931F93882339F487E3FC
:102F900096E061E77AE00E94C52B3BC090E00E947A
:102FA000B20824E630E040E050E00E94B92F122F32
:102FB000032FF42EE52E622F732F842F952F2AE0F6
:102FC00030E040E050E00E94B92F87E396E0BA017C
:102FD000A9012AE030E00E946D2C87E396E06EE2C2
:102FE0000E94A72B612F702F8F2D9E2D2AE030E09D
:102FF00040E050E00E94B92FAB01BC0187E396E0AE
:103000002AE030E00E946D2C87E396E063E70E949F
:10301000D92B1F910F91FF90EF900895FF920F937E
:103020001F93CF93DF9387E396E067E67AE00E94F1
:10303000862B8091B503813041F487E396E06EE4FE
:103040007AE00E94C52BFF246DC0823029F487E30B
:1030500096E067E37AE0F5CF843029F487E396E0E1
:1030600063E27AE0EECF853071F787E396E068E1BE
:103070007AE0E7CFCF2DD0E0C930D1051CF06F2D1D
:10308000685C02C06F2D6F5C87E396E00E94A72BFF
:1030900087E396E060E17AE00E94862BBE016F5FD5
:1030A0007F4F87E396E04AE050E00E94112D87E3CE
:1030B00096E065E07AE00E94862B8E010B541C4F4F
:1030C000D8011196EC91E032F8F487E396E068EFCE
:1030D00079E00E94862BF8018181803130F087E30E
:1030E00096E063E371E00E94382DCB54DC4F698198
:1030F00070E06F7070706F5F7F4F87E396E04AE01B
:1031000050E00E94242D0DC0F0E0EF70F070EE0F43
:10311000FF1FE75BFC4F6081718187E396E00E94AF
:103120003B2DF39480918A04F81608F4A3CF87E32B
:1031300096E06DED79E00E94862B8091CD030E9490
:10314000C11787E396E062EC79E00E94862B8091BC
:10315000CE030E94C11787E396E067EA79E00E94F8
:10316000862B8091CF030E94C11787E396E06CE81D
:1031700079E00E94862B4091C5035091C60360916F
:10318000C7037091C803411551056105710539F1F7
:1031900087E396E02AE030E00E947C2C87E396E00B
:1031A00069E579E00E94862B8091C9030E94E508B9
:1031B000AB01BC0187E396E02AE030E00E947C2C62
:1031C00087E396E065E379E00E94862B87E396E04B
:1031D0006091CA034AE050E00E94C72C06C087E312
:1031E00096E06CE279E00E94C52B87E396E06FE001
:1031F00079E00E94862B6091CB037091CC0387E32A
:1032000096E04AE050E00E94A12C87E396E062EF4E
:1032100078E00E94862B6091C403603150F470E026
:103220006F5F7F4F87E396E04AE050E00E94242DD5
:1032300006C087E396E069EE78E00E94C52B87E33D
:1032400096E06CEC78E00E94862B8091C30380FDB1
:1032500003C065E371E002C069E371E087E396E0D3
:103260000E943B2D87E396E06FEA78E00E94862B70
:103270008091C30382700E94840D87E396E060E929
:1032800078E00E94862B8091C30384700E94840D95
:1032900087E396E061E778E00E94862B8091C30384
:1032A00088700E94840DCDB7DEB7E5E00C941F3026
:1032B0001F93CF93DF9387E396E06BEB7BE00E9455
:1032C000862B4091D5035091D6036091D70370911E
:1032D000D80387E396E02AE030E00E947C2C87E365
:1032E00096E065EA7BE00E94862B4091D9035091DD
:1032F000DA036091DB037091DC0387E396E020E161
:1033000030E00E947C2C87E396E06FE87BE00E942F
:10331000862B87E396E06091DD034AE050E00E944F
:10332000C72C87E396E069E77BE00E94862B87E362
:1033300096E06091DE034AE050E00E94C72C87E3EC
:1033400096E063E67BE00E94862BCFEDD3E010E0B1
:1033500012C0112331F087E396E06DE371E00E9423
:10336000382D87E396E069914AE050E00E94B52C41
:103370001F5F183119F08881882359F787E396E099
:103380000E94AF2B87E396E06DE47BE00E94862BE2
:1033900087E396E06091F7034AE050E00E94C72C73
:1033A00087E396E068E37BE00E94862BE091F803D8
:1033B000F0E0E770F070EE0FFF1FE759FC4F6081FF
:1033C000718187E396E00E943B2D87E396E063E2FC
:1033D0007BE00E94862B8091F80390E088719070CA
:1033E0008830910589F0893091051CF4892B39F0DA
:1033F0001BC08031910569F04897B1F40FC087E395
:1034000096E06AE17BE00EC087E396E06EE07BE049
:1034100009C087E396E068E07BE004C087E396E0BC
:103420006EEF7AE00E94C52B87E396E06AEE7AE0C1
:103430000E94862B4091D1035091D2036091D30317
:103440007091D40387E396E02AE030E00E947C2C60
:1034500087E396E061ED7AE00E94862B8091A103DC
:1034600080710E94840D87E396E068EB7AE00E9409
:10347000862B8091A10380740E94840D87E396E0DF
:103480006FE97AE00E94862B8091A10380720E94EE
:10349000840D87E396E062E87AE00E94862B80ED57
:1034A00093E00E94F508AB01BC0187E396E02AE0B7
:1034B00030E00E946D2C87E396E06DE77AE00E9491
:1034C000862B80ED93E00E94F5089B01AC0160E43F
:1034D00072E48FE090E00E94B92F87E396E0BA0192
:1034E000A9012AE030E00E946D2C87E396E06AE7AC
:1034F0007AE00E94C52BDF91CF911F910895EF9242
:10350000FF920F931F938C0137E3E32E36E0F32EE7
:10351000C701612F70E04AE050E00E94902CC70183
:103520006EE20E94A72B24E0169507952A95E1F7F5
:103530000F701070C701B8014AE050E00E94902C53
:103540001F910F91FF90EF9008950F931F93CF93CA
:10355000DF93209101042F3FA9F587E396E061EF07
:1035600075E00E94862B80E793E00E947F1A87E334
:1035700096E060ED75E00E94862B80918B0490911F
:103580008C040E947F1A87E396E06DE975E00E9443
:10359000C52B87E396E06AE775E00E94C52B87E3B9
:1035A00096E062E675E00E94C52B87E396E06DE346
:1035B00075E00E94C52B87E396E00E94AF2B0E9426
:1035C0000E1869C012160CF066C0332727FD30951F
:1035D00080918A0490E0821793070CF45CC087E323
:1035E00096E068E275E00E94862B609101047727DF
:1035F00067FD709587E396E04AE050E00E94242D35
:1036000087E396E06DEF74E00E94862B10E008E2FD
:103610003AC0C12FD0E0CC0FDD1FC759DB4F288146
:1036200030E080910104992787FD90950197281734
:10363000390741F587E396E06FE371E00E94382D8A
:1036400087E396E0602F4AE050E00E94B52C87E3C4
:1036500096E063E471E00E94382DE981F0E0EF70BC
:10366000F070EE0FFF1FE75BFC4F6081718187E315
:1036700096E00E94382D87E396E067E471E00E94AF
:10368000382D0F5F1F5F80918904181710F287E3B0
:1036900096E00E94AF2BDF91CF911F910F9108957B
:1036A000ACE1B0E0E6E5FBE10C940030282F80911E
:1036B00001048F3F09F042C1822F90E0FC013A974C
:1036C000EF36F10508F033C1EC5CFF4F0C942D3060
:1036D00087E396E069E471E0AEC087E396E069E4D1
:1036E00071E00E943B2D1CC187E396E065E571E027
:1036F0000E943B2D85E78983DE011296E5EBF3E01E
:103700008BE101900D928150E1F7CE0101966CE1C1
:103710000E94C80F0E947F0C83E080939A0368EC9C
:1037200070E080E090E00E94122A80919A03843039
:1037300009F0FDC08FE70E94960A0E94AA0A8983B9
:10374000853509F0F4C087E396E06FED74E00E94E0
:10375000C52B87E396E061EC74E00E94C52B87E3FC
:1037600096E063EA74E0ACC087E396E06DE671E052
:103770000E943B2D89E68983CE01019661E00E947B
:10378000C80F0E947F0C83E080939A0368EC70E07E
:1037900080E090E00E94122A80919A03843009F020
:1037A000C6C08FE70E94960A0E94AA0A89838E01EA
:1037B0000E5F1F4FBDE1EB2EF12CEC0EFD1E0E94A3
:1037C000AA0AD8018D938D01AE15BF05C1F7A5EBEF
:1037D000B3E0FE0132968BE101900D928150E1F74A
:1037E0008981893409F0A3C087E396E065E874E035
:1037F0000E94C52B87E396E067E674E00E94C52B24
:1038000087E396E069E474E05BC087E396E067E8ED
:1038100071E00E943B2D8EEF8093010488C02052FE
:103820002750922F905380918A04891738F487E3A8
:1038300096E066E971E00E943B2D79C09093010407
:103840006FC084E18093010487E396E062E174E055
:1038500037C085E18093010487E396E06BED73E068
:103860002FC086E18093010487E396E064EA73E069
:1038700027C087E18093010487E396E06AE573E05F
:103880001FC088E18093010487E396E069E473E058
:1038900017C089E18093010487E396E065E373E054
:1038A0000FC08AE18093010487E396E060E273E051
:1038B00007C08BE18093010487E396E068EF72E034
:1038C0000E94C52B34C087E396E06EED72E00E9443
:1038D000C52B8091C30391E01DC087E396E068EC9F
:1038E00072E00E94C52B8091C30392E013C087E36E
:1038F00096E063EB72E00E94C52B8091C30394E0D5
:1039000009C087E396E068E972E00E94C52B8091C8
:10391000C30398E089278093C3038FEF809301044A
:103920000E94A51A04C087E396E00E94BA2E87E39E
:1039300096E00E94802E892BB1F762C1822F0E94EF
:103940000F17882309F45CC180916704882321F450
:103950008FEF809301044CC182E094E060E070E05E
:1039600040E050E00E94A2069B01AC01609101047E
:10397000862F992787FD9095A92FB92FFC013197A4
:10398000EB31F10508F024C1ED55FF4F0C942D30BB
:10399000E62FFF27E7FDF09580918A0490E08E17CF
:1039A0009F070CF415C1DA01C9010197A109B109FA
:1039B0008097A105B10548F0A8E2FA2E00E010E0DA
:1039C0006F010894C108D10825C0EB54FC4F822F29
:1039D00081508083E5C0612F70E0660F771F6759C3
:1039E0007B4FFB01808190E08C159D0591F48F2D1C
:1039F00090E0A0E0B0E082179307A407B50741F478
:103A0000F601EB54FC4FDB0111968C91818301E0B0
:103A1000F3941F5F809189041817E8F2BFC02F3F0D
:103A200031054105510511F008F0D2C02093CD03B6
:103A3000B7C02F3F31054105510511F008F0C8C04E
:103A40002093CE03ADC02F3F31054105510511F044
:103A500008F0BEC02093CF03A3C08091020480620F
:103A6000803719F583E094E060E070E040E050E0DA
:103A70000E94A2069B01AC01DC01CB010197A109C8
:103A8000B1090897A105B10508F0B5C0CA01B9018F
:103A900024ED30E340E050E00E94872F9B01AC0111
:103AA0002A5E3C4A4A46554E24C0863611F583E0CC
:103AB00094E060E070E040E050E00E94A2069B01CC
:103AC000AC01DC01CB010197A109B1090797A10560
:103AD000B10508F090C0CA01B90128EA31E640E01A
:103AE00050E00E94872F9B01AC01245E3C434E4670
:103AF000544E211531054105510561F0DA01C90126
:103B000080509447AB48B24381509A45A246B24098
:103B100008F05EC02093C5033093C6034093C703EB
:103B20005093C8033DC02F3F31054105510511F0A9
:103B300008F04EC02093C90333C0DA01C9010197D0
:103B4000A109B1098F3F9105A105B10508F040C059
:103B50002093CA0325C0DA01C901845C9940A040C2
:103B6000B0408D549D41A040B04030F43093CC0320
:103B70002093CB0301E001C000E021153105410590
:103B8000510511F48FEF07C0213131054105510571
:103B900028F4822F81508093C40302C00023C1F017
:103BA000809168048823D1F48091D9039091DA033D
:103BB000A091DB03B091DC030196A11DB11D8093A0
:103BC000D9039093DA03A093DB03B093DC0306C020
:103BD00087E396E068EA71E00E943B2D0E9405179A
:103BE0008FEF8093010487E396E06AE00E94D92B6F
:103BF0000E94A51A05C021E030E040E050E07ECFF1
:103C00006C96E8E00C941C3087E396E06CE472E07C
:103C10000E94C52B87E396E064E372E00E94C52B07
:103C200087E396E00E94802E892B31F087E396E0AF
:103C30000E94BA2E0E94501B0E941C15823019F05F
:103C4000833069F405C087E396E066E172E004C062
:103C500087E396E06FEF71E00E94C52B08958FEF28
:103C600080930104109268040E94A51A0CC087E397
:103C700096E00E94802E892B31F087E396E00E9427
:103C8000BA2E0E94501B809101048E3F81F7089547
:103C900080910104992787FD9095A92FB92FFC01E8
:103CA0003196EB30F10508F074C0E254FF4F0C94EC
:103CB0002D3087E396E064E678E00E94C52B80E72C
:103CC00093E00E947F1A87E396E06CE478E00E941C
:103CD000C52B87E396E067E278E00E94C52B87E377
:103CE00096E06DEF77E00E94C52B87E396E06CEDE0
:103CF00077E00E94C52B87E396E06FEA77E00E94A9
:103D0000C52B87E396E069E877E00E94C52B87E33F
:103D100096E065E677E00E94C52B87E396E06EE3C8
:103D200077E00E94C52B87E396E00E94AF2B0E94AC
:103D300058192FC087E396E061E277E028C087E357
:103D400096E06CEF76E023C087E396E067EE76E0DE
:103D50001EC087E396E068EC76E019C087E396E042
:103D600064E876E014C087E396E06FE676E00FC083
:103D700087E396E06AE576E00E94C52B87E396E04C
:103D800064E176E004C087E396E06EEF75E00E94A0
:103D9000C52B6AE070E080E090E00E94122A04C027
:103DA00087E396E00E94BA2E87E396E00E94802E79
:103DB000892BB1F70895A2E2B0E0E1EEFEE10C94A8
:103DC000F62F8E010F5F1F4F80E1D8011D928A955B
:103DD000E9F787E396E066EC71E00E943B2D0E94D4
:103DE000C81520E034E74BE852E32F8F38A349A3EE
:103DF0005AA380E09EECADEEB4E38B8F9C8FAD8F29
:103E0000BE8F24EF31E040E050E02F8B388F498F98
:103E10005A8F30E5C32E33ECD32EE12CF12C412CFC
:103E200024E7522E2BE8622E22E3722E8824992456
:103E3000540133241E8A1D8A198A1A8A1B8A1C8AF5
:103E4000FFC087E396E00E94BA2E8434B9F085342F
:103E500030F48332B9F18C3209F0CCC044C08335E0
:103E600009F0C8C02F8D38A149A15AA1C901DA01B2
:103E70002C013D01882499245401E2C087E396E097
:103E800064E40E94A72B87E396E040E054E76BE8E8
:103E900072E32AE030E00E94DB2C87E396E06CE2DC
:103EA0000E94A72B87E396E040E05EEC6DEE74E3A2
:103EB0002AE030E00E94DB2C87E396E06CE20E946F
:103EC000D92BBEC019821A821B821C821D821E82BF
:103ED0001F82188619861A861B861C861D861E86DA
:103EE0001F86188A3AC0339434E0331609F0A8C00C
:103EF00069817A818B819C8128EE33E040E050E03B
:103F00000E94872F6F8F78A389A39AA36D817E81EA
:103F10008F8198850E94872F6B8F7C8F8D8F9E8FCE
:103F200089859A85AB85BC858F8B988FA98FBA8F31
:103F30006D857E858F8598890E94872F6B017C0116
:103F400090E2C9169EE4D90690E0E90690E0F906F1
:103F500030F48CE162E30E94C00A332471C0A0E314
:103F6000CA16A5E7DA06A0E0EA06A0E0FA0618F409
:103F70008CE162E2F0CFB0E4CB16BCE9DB06B0E046
:103F8000EB06B0E0FB0618F48CE166E2E4CFE0E576
:103F9000CE16E3ECDE06E0E0EE06E0E0FE0618F406
:103FA0008CE162E1D8CFF0E6CF16FAEEDF06F0E062
:103FB000EF06F0E0FF0618F48CE165E1CCCF20E7D6
:103FC000C21621E1D20621E0E20620E0F20618F452
:103FD0008CE161E0C0CF30EAC31636E8D30631E0A9
:103FE000E30630E0F30618F48CE163E0B4CF8CE133
:103FF00065E0B1CF90ED292E280E49E0421500F181
:10400000032D10E0000F111F000F111F81E090E041
:104010008C0F9D1F080F191FD8016D917D918D91F7
:104020009C912AE030E040E050E00E94872F620D32
:10403000711D811D911DF8016083718382839383BB
:1040400087E396E00E94802E892B09F0FACE811436
:104050009104A104B10489F4C301B2010E94360B9A
:1040600061E070E080E090E00E94122AFFEFFE8B9A
:104070001D8A198A1A8A1B8A1C8A2F89388D498DB4
:104080005A8D82169306A406B506E0F40E94E10A52
:1040900029893A894B895C89280F311D411D511DA1
:1040A000298B3A8B4B8B5C8B3D89381708F48D8BB1
:1040B0004E89841708F48E8B0894811C911CA11CD6
:1040C000B11C56C0C301B20128EE33E040E050E01D
:1040D0000E94B92F87E396E0BA01A9012AE030E0F7
:1040E0000E946D2C87E396E06CE20E94A72B87E389
:1040F00096E06D894AE050E00E94B52C87E396E097
:104100006CE20E94A72B69897A898B899C89A50119
:1041100094010E94B92F87E396E0BA01A9012AE031
:1041200030E00E946D2C87E396E06CE20E94A72BA2
:1041300087E396E06E894AE050E00E94B52C87E361
:1041400096E06CE20E94D92B4C0C5D1C6E1C7F1C0F
:104150008B8D9C8DAD8DBE8D84159505A605B705FF
:1041600020F44F8C58A069A07AA088249924540187
:104170002F8D38A149A15AA1285E334040405040BC
:1041800009F05ECFA296E2E10C941230AAE5B0E00D
:10419000ECECF0E20C9402308B017A018B3009F4E4
:1041A00026C18C3040F5853009F484C0863080F417
:1041B000823009F459C0833020F4813009F052C2B2
:1041C00042C0833009F461C0843009F04BC265C03D
:1041D000883009F49DC0893038F4863009F486C0EF
:1041E000873009F03FC28CC0893009F499C08A3009
:1041F00009F038C2C9C0893609F484C18A3680F40E
:10420000863609F42FC1873620F4853609F02AC294
:1042100010C1873609F43FC1883609F023C243C173
:104220008C3609F4C6C18D3638F48A3609F475C166
:104230008B3609F017C2B1C18D3609F4EEC1873C47
:1042400009F010C202C281E069E270E00E948011B0
:1042500000ED13E0F80181918F010E946911F3E0F4
:10426000093F1F07B9F706C282E06BE170E00E94C8
:10427000801105EB13E0F80181918F010E94691113
:10428000F3E0003D1F07B9F7F5C183E061E070E09E
:104290000E9480110E941C15EBC184E061E070E077
:1042A0000E94801181E00E9469110E9462110E94A7
:1042B000DB1EE2C16091890470E0660F771F85E024
:1042C0000E94801100E010E008C0F801E759FB4FA0
:1042D00080810E9469110F5F1F4F8091890490E0D7
:1042E000880F991F0817190780F3C4C186E062E0A0
:1042F00070E00E94801180E793E00E947711BAC1BC
:1043000087E061E070E00E94801180918A04B0C172
:1043100088E061E070E00E94801180919B03A8C159
:1043200086E68983CE01019661E00E94C80F0E9453
:104330007F0C83E080939A0368EC70E080E090E06B
:104340000E94122A80919A038430E1F48FE70E9440
:10435000960A0E94AA0A8983863471F489E060E291
:1043600070E00E94801110E00E94AA0A0E94691168
:104370001F5F1032C9F77EC189E061E070E00E94E2
:104380008011C9C089E06FC18AE069E170E00E94D4
:10439000801181E080939C038091A105882351F0D6
:1043A0008091A1039091A203A091A303B091A403D3
:1043B000806809C08091A1039091A203A091A303FA
:1043C000B091A4038F778093A1039093A203A0934D
:1043D000A303B093A4030CE913E0F80181918F01CA
:1043E0000E946911F3E0053B1F07B9F743C18BE059
:1043F00061E270E00E9480118091BE048F3F39F02D
:104400008091BE048F5F8093BE04815002C0809172
:10441000BE040E94691110E0F894812F0E949F1140
:104420000E94190A0E94771178941F5F1031A1F73A
:1044300021C185E661E070E00E948011093211051A
:1044400009F015C120E030E0F901E053FC4FD7013D
:10445000A20FB31F8C9180832F5F3F4F293231050C
:1044600099F759C086E661E070E00E9480110B3137
:10447000110509F0FCC020E030E0F901EB54FC4FDD
:10448000D701A20FB31F8C9180832F5F3F4F2B3139
:10449000310599F740C087E661E070E00E94801125
:1044A0000E94C71638C088E661E070E00E94801163
:1044B00085E78A83DE011396E5EBF3E08BE101905B
:1044C0000D928150E1F7CE0102966CE10E94C80F77
:1044D0000E947F0C83E080939A0360E273E080E0A7
:1044E00090E00E94122A80919A03843009F0BFC0A4
:1044F0008FE70E94960A0E94AA0A8A83853509F0EE
:10450000B6C009C089E661E070E00E9480110E9497
:104510004D080E94920881E0ABC08AE661E070E03D
:104520000E94801189E68E8FCE014E9661E00E9436
:10453000C80F0E947F0C83E080939A0360E273E0CF
:1045400080E090E00E94122A80919A03843009F062
:104550008EC08FE70E94960A0E94AA0A8E8F8E0153
:10456000015E1F4F4AE3E42EF12CEC0EFD1E0E946B
:10457000AA0AF80181938F01EE15FF05C1F7A5EB9B
:10458000B3E0FE017F968BE101900D928150E1F73F
:104590008E8D893409F06BC0BECF8BE661E070E090
:1045A0000E948011F70180810E94F5160E94D016AA
:1045B000B2CF8CE661E070E00E94801100321105FC
:1045C00071F487E68AAFDE01DB96F70180E20190A5
:1045D0000D928150E1F7CE01CA9661E205C087E4F1
:1045E0008AAFCE01CA9661E00E94C80F0E947F0C7C
:1045F00083E080939A036CE474E080E090E00E9492
:10460000122A80919A03843091F58FE70E94960ACE
:104610000E94AA0A873459F57ECF8DE661E070E0EA
:104620000E9480110931110511F520E030E0F901F7
:10463000E456FC4FD701A20FB31F8C9180832F5FEC
:104640003F4F2931310599F766CF87EC61E070E083
:104650000E94801181E00E9469110E9462111092F3
:10466000FF030AC08AEC61E070E00E94801180E0E4
:104670000E9469110E946211C65ADF4FE6E00C9455
:104680001E30A0E0B0E0E7E4F3E20C94FE2F84E0FB
:10469000A82E06E0B02E15E0C12E05E315E0B4E625
:1046A000DB2EA2E0EA2EF3E0FF2EA1C087E396E026
:1046B0000E94BA2E982F8093A00580919F05833089
:1046C00021F1843028F4813099F08230B8F409C0A7
:1046D000853009F448C0853020F1863009F087C064
:1046E0005FC0953B09F083C081E080939F057FC048
:1046F000923609F07AC0E0929F0579C090939E05AA
:1047000090939D05F0929F0572C090939B05109227
:104710009C0580919D05892780939D05A0929F050A
:1047200066C0D92FC0E020919B0530919C052C2BB1
:104730003D2B30939C0520939B0580919D058927F7
:1047400080939D05C0929F052536310508F44FC022
:104750008CEC61E070E00E94801181E00E946911A0
:104760000E94621142C02091990530919A05F90189
:10477000EB5CFA4F908380919D05892780939D057E
:104780002F5F3F4F30939A052093990580919B05A9
:1047900090919C052817390750F1B0929F0527C0CA
:1047A00080919D05891759F46091990570919A053A
:1047B00080919E0545E355E00E94C6200DC08BEC1C
:1047C00062E070E00E94801180919E050E94691154
:1047D000809100040E946911F8018D2D11928A9533
:1047E000E9F710929A051092990510929F0587E3B8
:1047F00096E00E94802E892B09F058CFCDB7DEB706
:10480000EAE00C941A3081E08093FF0308C087E34C
:1048100096E00E94802E892B11F00E944123809106
:10482000FF038823A1F70895A0E0B0E0EAE1F4E2F5
:104830000C9401300E94EC296115710581059105E8
:10484000C9F30E9499061092D9031092DA031092CC
:10485000DB031092DC03DD24E090D903F090DA034F
:104860000091DB031091DC03102F0F2DFE2CEE24A2
:104870000E9494062FEF30E040E050E00E94DB2FD2
:10488000E60EF71E081F191FE092D903F092DA0313
:104890000093DB031093DC03D39444E0D416E1F6D9
:1048A000CFEDD3E000E010E090E1E92E97E2F92EA1
:1048B0004EC00F5F19F40E944D084DC00E9494062F
:1048C00022E330E040E050E00E94DB2F6F5FEFED2D
:1048D000F3E090E004C08191861759F39F5F911730
:1048E000D0F38091DE0390E08E9D90018F9D300D7E
:1048F0009E9D300D1124862F90E0AC01249FC001B5
:10490000259F900D349F900D1124AA2797FDA09507
:10491000BA2F2091D5033091D6034091D7035091FF
:10492000D803820F931FA41FB51F20919D033091C0
:104930009E0340919F035091A003281739074A070F
:104940005B0708F4B6CF69931F5F183121F08881A7
:10495000882309F0AECFCDB7DEB7E7E00C941D3069
:104960001F93109101041F3F09F0F1C0893409F42D
:1049700067C08A3428F5883309F479C0893368F42C
:10498000803309F486C0813308F06FC08B3109F49D
:104990004DC0813209F0D5C03DC0813409F49AC0C0
:1049A000823438F4893309F472C0803409F0C9C004
:1049B00031C0823409F4A1C0863409F0C2C052C0AB
:1049C000823609F49AC0833690F4883579F18935B6
:1049D00038F4823509F43FC0833509F0B2C01FC0F6
:1049E0008A3509F4A9C0813609F0ABC073C082379B
:1049F00091F1833730F48636A9F1893609F0A1C0E8
:104A00001FC0883799F08A3709F496C0833709F0B8
:104A100098C005C087E396E069E471E019C00E9480
:104A2000C71687E396E063ED71E006C00E94D016DA
:104A300087E396E06DEE71E00E943B2D8EEF7FC024
:104A40000E944D080E94920887E396E06CE072E0B5
:104A50000E943B2D76C00E94142487E396E065E215
:104A600072E0F6CF0E9478176CC0805368C087E36D
:104A700096E06CEE71E00E94C52B9091F803892FAF
:104A8000885F8871977E892B8093F80320C089E026
:104A900056C087E396E069ED71E00E94C52B8091D6
:104AA000A1039091A203A091A303B091A40320E1DC
:104AB00030E040E050E082279327A427B527809379
:104AC000A1039093A203A093A303B093A403109314
:104AD000010437C087E396E063EC71E00E94C52BC8
:104AE0008091A1039091A203A091A303B091A4038C
:104AF00020E430E040E050E012C087E396E062EB53
:104B000071E00E94C52B8091A1039091A203A09116
:104B1000A303B091A40320E230E040E050E08227FC
:104B20009327A427B5278093A1039093A203A09372
:104B3000A303B093A40302C00E94041E8FEF8093CE
:104B40000104809101048E3F09F4DDC0D4C00E94AD
:104B50000F17882309F4D7C080916704882321F4B4
:104B60008FEF80930104C7C082E094E060E070E0C2
:104B700040E050E00E94A2069B01AC01809101043C
:104B8000992787FD9095A92FB92FFC013197E9301E
:104B9000F10508F08CC0E753FF4F0C942D30DA017B
:104BA000C90181509447AB48B2438F5F9945A246F3
:104BB000B24008F07CC02093D5033093D6034093D5
:104BC000D7035093D8039AC02093D9033093DA03C4
:104BD0004093DB035093DC0381E0809368048EC034
:104BE000283031054105510508F061C02093DD03EF
:104BF00085C0DA01C9010197A109B1090A97A10588
:104C0000B10508F054C02093DE0378C082E094E040
:104C10006DE371E00E94BE0710E00EC0183130F461
:104C2000E12FF0E0E053FC4F87871F5F80E090E0CA
:104C30006DE371E00E94BE07009759F00E94A00743
:104C4000009761F706C0E12FF0E0E053FC4F1786B4
:104C50001F5F1831C0F352C02530310541055105A1
:104C600030F52093F7034AC0DA01C9010197A10981
:104C7000B1090697A105B105D0F48091F803887FAA
:104C8000822B8093F8033AC0DA01C9010197A10988
:104C9000B1098050924CA140B04048F42093D10318
:104CA0003093D2034093D3035093D40327C087E3B8
:104CB00096E068EA71E00E943B2D13C08091D90311
:104CC0009091DA03A091DB03B091DC030196A11D62
:104CD000B11D8093D9039093DA03A093DB03B093C3
:104CE000DC030E9405178FEF8093010487E396E0B1
:104CF0006AE00E94D92B0E94481E05C0809168047A
:104D00008823E1F2EECF1F9108958FEF8093010485
:104D1000109268040E94481E0CC087E396E00E942F
:104D2000802E892B31F087E396E00E94BA2E0E94F4
:104D3000B024809101048E3F81F76AE070E080E04A
:104D400090E00E94122A04C087E396E00E94BA2EE7
:104D500087E396E00E94802E892BB1F70895AAE29E
:104D6000B0E0E5EBF6E20C94FB2F0E94DE297B011C
:104D70008C0181E00E94A00B04C087E396E00E94B2
:104D8000BA2E87E396E00E94802E892BB1F75E98B9
:104D90004098DD24D39452E6752E42E0842E912C67
:104DA0008C0E9D1E5E010894A11CB11C33E0C32E25
:104DB0000E94DE2920E030E06E197F09800B910B04
:104DC000693C71058105910510F021E030E08D2DE1
:104DD00090E028233923232BA9F10E94DE297B01AF
:104DE0008C015D9A419A80ED97E00E94D3117982FF
:104DF000D401E0EDF3E089E201900D928150E1F7FA
:104E0000C5016AE20E94C80F5D98419880E090E079
:104E10000E94D311C0929A030E947F0C62E370E05B
:104E200080E090E00E94122A80919A03843051F42D
:104E3000C0929A038FE70E94960A0E94AA0A8234BF
:104E400009F4DD2482E10E94102B892B69F5DD2411
:104E5000D3942AC05E9A409A5D9A419A87E396E07D
:104E60000E94BA2E8D30910569F08E3091051CF4A8
:104E70000A97B1F407C08332910569F08234910535
:104E800079F40CC087E396E064EA71E00E94C52BD8
:104E90000E94852605C00E94DB1E02C00E940324DA
:104EA0005E9840985D98419887E396E00E94802E36
:104EB000892B09F47DCFCECF8F929F92AF92BF9274
:104EC000CF92DF92EF92FF920F931F9382E10E94A5
:104ED000102B892B09F083C068EC70E080E090E033
:104EE0000E94122A80E090E00E94D3110E94DE29E5
:104EF0005B016C0160ECE62E62E1F62E012D112DB6
:104F0000EA0CFB1C0C1D1D1D06C082E10E94102B2B
:104F1000892B09F062C00E94DE296E157F0580078B
:104F2000910798F382E10E94102B892B09F055C05C
:104F300080ED97E00E94D3110E94DE297B018C0155
:104F400099249394882488E496E2A0E0B0E0A80E27
:104F5000B91ECA1EDB1E29C0AE14BF04C006D1068E
:104F600038F480ED97E00E94D311882483941DC00B
:104F70000E94DE296E197F09800B910B693C710537
:104F80008105910590F00E94DE297B018C0180E073
:104F9000992009F481E0982E882319F480E090E0AC
:104FA00002C080ED97E00E94D31182E10E94102B95
:104FB000892B91F280E090E00E94D311882049F083
:104FC00080919B038F5F83700E94F5160E94D0161C
:104FD00006C00E9414240E94C7160E94AF261F918B
:104FE0000F91FF90EF90DF90CF90BF90AF909F9088
:104FF0008F90089580E06DEF77E042E050E00E94EE
:1050000019290895EF92FF920F931F9380E00E9459
:1050100019080E94BE1186E061E00E94712A85E0B5
:1050200061E00E94712A8EE061E00E94712A8FE0A7
:1050300061E00E94712A82E160E00E94712A88E0AA
:1050400060E00E94712A88E061E00E94DD2A0E94EF
:10505000E61487E396E040E052EC61E070E00E94E5
:10506000F92D0E94E8160E94D0160E945F0D8FEF66
:105070008093BE040E94FA2778940E94DE297B0167
:105080008C018091BE048F3F09F0C8C00E94DE29C8
:105090006E197F09800B910B605D774080409040D6
:1050A00008F0BCC0EECF87E396E00E94BA2E87E3FB
:1050B00096E00E94802E892BB1F787E396E062E4A8
:1050C00072E00E94382D80E793E00E947F1A87E308
:1050D00096E069E572E00E94382D87E396E065E08E
:1050E00070E04AE050E00E94242D62E370E080E02E
:1050F00090E00E94122A87E396E00E94802E049797
:105100000CF187E396E00E94BA2E82349105D1F427
:1051100087E396E00E94BA2E8E34910599F487E3D6
:1051200096E00E94BA2E8434910561F487E396E0FC
:105130000E94BA2E819731F480E090E00E94D31152
:105140000E94AF264091D1035091D2036091D303C6
:105150007091D403DB01CA010197A109B109049739
:10516000A105B10568F44093BF04433029F040E045
:1051700052EC61E070E004C040EA56E861E070E0A3
:1051800087E396E00E94F92D0E945C275E98409884
:1051900080E090E00E94D3110E945F0D80E00E94A9
:1051A000A00B8091A4040E94CB0A0E947F0C109255
:1051B000290510922A0510922B0510E015C062E314
:1051C00070E080E090E00E94122A80ED97E00E945B
:1051D000D31162E370E080E090E00E94122A80E048
:1051E00090E00E94D3111F5F80919B03811738F7D5
:1051F0008091F80390E084FF09C020E088719070EE
:10520000489709F421E0822F0E94FD148FE00E944C
:1052100019081F910F91FF90EF90089580ED97E08E
:105220000E94D31182E161E00E94DD2A5E9A409AD9
:105230003ECF823000F5E82FF0E0EE0FFF1FEE5575
:10524000FA4F71836083882319F08130A1F408C07C
:10525000809169008C7F842B80936900E89A08957F
:1052600080916900440F551F440F551F837F842B85
:1052700080936900E99A08951F920F920FB60F92DA
:1052800011242F933F934F935F936F937F938F934B
:105290009F93AF93BF93EF93FF938091A20590915B
:1052A000A305892B29F0E091A205F091A3050995AA
:1052B000FF91EF91BF91AF919F918F917F916F91EE
:1052C0005F914F913F912F910F900FBE0F901F90C4
:1052D00018951F920F920FB60F9211242F933F93A0
:1052E0004F935F936F937F938F939F93AF93BF93EE
:1052F000EF93FF938091A4059091A505892B29F048
:10530000E091A405F091A5050995FF91EF91BF915A
:10531000AF919F918F917F916F915F914F913F914D
:105320002F910F900FBE0F901F9018951F920F9204
:105330000FB60F9211242F933F938F939F93AF93A8
:10534000BF938091AA059091AB05A091AC05B09157
:10535000AD053091AE050196A11DB11D232F2D5F26
:105360002D3720F02D570196A11DB11D2093AE05BC
:105370008093AA059093AB05A093AC05B093AD05BF
:105380008091A6059091A705A091A805B091A905C7
:105390000196A11DB11D8093A6059093A705A0932A
:1053A000A805B093A905BF91AF919F918F913F91AF
:1053B0002F910F900FBE0F901F9018958FB7F894F4
:1053C0002091AA053091AB054091AC055091AD05F7
:1053D0008FBFB901CA0108959FB7F8942091A6051F
:1053E0003091A7054091A8055091A90586B5A89BC5
:1053F00006C08F3F21F02F5F3F4F4F4F5F4F9FBF42
:10540000542F432F322F2227280F311D411D511DAC
:1054100082E0220F331F441F551F8A95D1F7B9012F
:10542000CA010895EF92FF920F931F93CF93DF93DA
:105430007B018C010E94EC29EB010EC00E94EC293B
:105440006C1B7D0B685E7340C8F30894E108F1089B
:1054500001091109C851DC4FE114F10401051105DE
:1054600069F7CDB7DEB7E6E00C941E30789484B5CA
:10547000826084BD84B5816084BD85B5826085BD50
:1054800085B5816085BDEEE6F0E080818160808336
:10549000E1E8F0E010828081826080838081816019
:1054A0008083E0E8F0E0808181608083E1EBF0E0E0
:1054B000808184608083E0EBF0E080818160808384
:1054C000EAE7F0E08081846080838081826080836D
:1054D0008081816080838081806880831092C10098
:1054E0000895CF93DF93482F50E0CA018D5F934F0B
:1054F000FC0134914151544FFA018491882369F1A0
:1055000090E0880F991FFC01EF52F44FA591B491E0
:10551000FC01E552F44FC591D491662351F42FB7A5
:10552000F8948C91932F909589238C93888189236B
:105530000BC0623061F42FB7F8948C91932F909543
:1055400089238C938881832B88832FBF06C09FB7C4
:10555000F8948C91832B8C939FBFDF91CF9108950A
:10556000833071F0843028F48130A1F0823021F54D
:1055700014C08630B1F08730D1F08430E9F404C033
:10558000809180008F7703C0809180008F7D809311
:105590008000089584B58F7702C084B58F7D84BD67
:1055A00008958091B0008F778093B0000895809126
:1055B000B0008F7D8093B0000895FF920F931F93EA
:1055C000F62E482F50E0CA01895E934FFC012491CA
:1055D000CA018D5F934FFC0114914151544FFA0160
:1055E00004910023C9F0222319F0822F0E94B02ACF
:1055F000E02FF0E0EE0FFF1FE552F44FA591B491BC
:105600009FB7F894FF2021F48C911095812302C05C
:105610008C91812B8C939FBF1F910F91FF900895C8
:105620000F931F93482F50E0CA01895E934FFC01EE
:105630002491CA018D5F934FFC0104914151544F55
:10564000FA011491112319F420E030E015C022234F
:1056500019F0822F0E94B02A812F90E0880F991FA5
:105660008B51944FFC01A591B4918C9120E030E0D6
:10567000802311F021E030E0C9011F910F910895BE
:10568000982F8E3008F09E50977080914803829535
:10569000880F880F807C892B80937C0080917A0012
:1056A000806480937A0080917A0086FDFCCF2091FF
:1056B000780040917900942F80E030E0282B392B3E
:1056C000C9010895A0E0B0E0E8E6FBE20C940030E8
:1056D0007C016B018A01C0E0D0E00FC0D6016D9162
:1056E0006D01D701ED91FC910190F081E02DC70192
:1056F0000995C80FD91F015010400115110571F708
:10570000CE01CDB7DEB7E8E00C941C30EF92FF92EB
:105710000F931F93CF93DF937C018B01C0E0D0E008
:10572000F8010F5F1F4F6491662359F0D701ED9187
:10573000FC910190F081E02DC7010995C80FD91F98
:10574000EFCFCE01CDB7DEB7E6E00C941E30DC0122
:10575000ED91FC910190F081E02D09950895EF9273
:10576000FF920F931F938C016DE00E94A72B7C0189
:10577000C8016AE00E94A72B9C012E0D3F1DC901A4
:105780001F910F91FF90EF900895EF92FF920F936A
:105790001F937C010E94862B8C01C7010E94AF2BB6
:1057A0009C01200F311FC9011F910F91FF90EF90B5
:1057B0000895EF92FF920F931F937C010E94A72BF5
:1057C0008C01C7010E94AF2B9C01200F311FC90122
:1057D0001F910F91FF90EF900895CF93DF93EC010D
:1057E0006115710519F420E030E00FC0DB010D9068
:1057F0000020E9F71197A61BB70BE881F981028019
:10580000F381E02DAD0109959C01C901DF91CF9194
:1058100008954F925F927F928F929F92AF92BF9224
:10582000CF92DF92EF92FF920F931F93DF93CF936C
:10583000CDB7DEB7A1970FB6F894DEBF0FBECDBFD0
:105840002C01742ECB01223008F42AE019A231E297
:10585000C32ED12CCC0EDD1E822E9924AA24BB246B
:10586000672D752FA50194010E94B92F79018A0136
:10587000C801B701A50194010E94872F472D461B3F
:105880000894C108D1084A3010F4405D01C0495C59
:10589000F6014083E114F1040105110521F07E2C8D
:1058A0005F2DC801DDCFC201B6010E94ED2BA1968C
:1058B0000FB6F894DEBF0FBECDBFCF91DF911F9121
:1058C0000F91FF90EF90DF90CF90BF90AF909F909F
:1058D0008F907F905F904F900895DC0121153105E6
:1058E00041F4ED91FC910190F081E02D642F099538
:1058F00008950E94092C0895EF92FF920F931F9331
:105900007C010E946D2C8C01C7010E94AF2B9C0171
:10591000200F311FC9011F910F91FF90EF90089543
:10592000EF92FF920F931F939A017B0100E010E02A
:10593000B801A7010E946D2C1F910F91FF90EF906D
:105940000895EF92FF920F931F937C010E94902C79
:105950008C01C7010E94AF2B9C01200F311FC90190
:105960001F910F91FF90EF900895EF92FF920F9388
:105970001F939A01E62EFF2400E010E0B801A70172
:105980000E946D2C1F910F91FF90EF900895EF9260
:10599000FF920F931F937C010E94B52C8C01C701CD
:1059A0000E94AF2B9C01200F311FC9011F910F9145
:1059B000FF90EF900895A0E0B0E0E1EEFCE20C94DF
:1059C0000030EC016A017B012115310541F4E881C9
:1059D000F9810190F081E02D642F09951BC02A30D8
:1059E0003105B1F477FF13C06DE20E94A72B8C0143
:1059F00044275527BA014C195D096E097F09CE016C
:105A00002AE00E94092C9C01200F311F04C02AE0CB
:105A10000E94092C9C01C901CDB7DEB7E8E00C94C7
:105A20001C30EF92FF920F931F937B019A01002786
:105A3000F7FC0095102FB801A7010E94DB2C1F91E5
:105A40000F91FF90EF900895EF92FF920F931F93A5
:105A50007C010E94112D8C01C7010E94AF2B9C017B
:105A6000200F311FC9011F910F91FF90EF900895F2
:105A70000E94ED2B0895EF92FF920F931F937C01EC
:105A80000E94382D8C01C7010E94AF2B9C01200F72
:105A9000311FC9011F910F91FF90EF900895089554
:105AA0001F920F920FB60F9211242F933F934F9393
:105AB0008F939F93EF93FF938091C00082FD1DC051
:105AC0004091C6002091EF053091F0052F5F3F4FC8
:105AD0002F7330708091F1059091F20528173907E6
:105AE00071F0E091EF05F091F005E155FA4F408338
:105AF0003093F0052093EF0502C08091C600FF911E
:105B0000EF919F918F914F913F912F910F900FBEE9
:105B10000F901F9018951F920F920FB60F9211249D
:105B20002F933F938F939F93EF93FF93209133068F
:105B30003091340680913506909136062817390742
:105B400031F48091C1008F7D8093C10014C0E09139
:105B50003506F0913606ED50FA4F208180913506DA
:105B60009091360601968F739070909336068093CD
:105B700035062093C600FF91EF919F918F913F9141
:105B80002F910F900FBE0F901F901895A0E0B0E0DE
:105B9000ECECFDE20C94FC2FFC011382128288EEE7
:105BA00093E0A0E0B0E084839583A683B7838BE87D
:105BB00093E0918380837587648757874687318B0D
:105BC000208B138B028BF58AE48AD78AC68AB18E22
:105BD000A08E938E828E8F85848F8889858F898908
:105BE000868F8A89878F8B8980A32096ECE00C941E
:105BF0001830AF92BF92DF92EF92FF920F931F93F4
:105C0000CF93DF93EC017A018B01DD24403081EEEC
:105C1000580780E0680780E0780711F0DD24D3940E
:105C200091E0A92EB12CEC89FD89DD2069F0C50138
:105C300008A002C0880F991F0A94E2F7808360E0F1
:105C400079E08DE390E005C0108260E874E88EE1B1
:105C500090E0A80197010E94B92F215030404040A8
:105C60005040569547953795279580E12030380765
:105C700020F0DD2011F0DD24D6CFE889F9893083CA
:105C8000EA89FB89208319A2EE89FF89408121E0FE
:105C900030E0C9010C8C02C0880F991F0A94E2F70A
:105CA000482B4083EE89FF894081C9010D8C02C0D9
:105CB000880F991F0A94E2F7482B4083EE89FF89E9
:105CC0004081C9010E8C02C0880F991F0A94E2F727
:105CD000482B4083EE89FF8980810F8C02C0220F00
:105CE000331F0A94E2F7209528232083DF91CF9178
:105CF0001F910F91FF90EF90DF90BF90AF900895AC
:105D0000DC011C96ED91FC911D97E05CFF4F219109
:105D1000319180819181281B390B2F733070C9011B
:105D2000089587E396E00E94802E892B11F00E944F
:105D30004F2D0895DC011C96ED91FC911D97E05CC0
:105D4000FF4F20813181E054F040DF01AE5BBF4F57
:105D50008D919C9111972817390719F42FEF3FEF78
:105D600007C08D919C91E80FF91F8081282F30E0AA
:105D7000C9010895DC011C96ED91FC911D97E05C32
:105D8000FF4F20813181E054F040DF01AE5BBF4F17
:105D90008D919C9111972817390719F42FEF3FEF38
:105DA00010C08D919C911197E80FF91F20818D9162
:105DB0009C91119701968F73907011969C938E937E
:105DC00030E0C9010895DC0191968C919197882368
:105DD00039F05496ED91FC915597808186FFF9CF6B
:105DE00091961C920895CF93DF93EC01EE85FF8589
:105DF000E05CFF4F20813181E054F0402F5F3F4F46
:105E00002F733070DF01AE5BBF4F8D919C91119766
:105E100028173907D1F3E05CFF4F80819181E0546E
:105E2000F040E80FF91F6083EE85FF85E05CFF4FCF
:105E300031832083EE89FF89208181E090E00F8CFF
:105E400002C0880F991F0A94E2F7282B208381E073
:105E500089A3EC89FD8980818064808381E090E062
:105E6000DF91CF9108958F929F92AF92BF92CF9280
:105E7000DF92EF92FF920F931F9300D000D00F920A
:105E8000EDB7FEB7319684E0ADB7BEB711968C93EF
:105E900083E0818387E0828385E0838381E084835C
:105EA00087E396E06FEA75E043EF55E025EC30E0DC
:105EB00004EC10E0B0ECEB2EF12CA1ECCA2ED12CAE
:105EC000F2ECAF2EB12CE6EC8E2E912C0E94C62D5A
:105ED0000F900F900F900F900F901F910F91FF90C8
:105EE000EF90DF90CF90BF90AF909F908F900895EC
:105EF000CF93DF930E94362A0E940228C1E9DEE296
:105F00000E9415122097E1F30E94912EF9CF629F13
:105F1000D001739FF001829FE00DF11D649FE00DA1
:105F2000F11D929FF00D839FF00D749FF00D659F02
:105F3000F00D9927729FB00DE11DF91F639FB00D01
:105F4000E11DF91FBD01CF011124089597FB092E12
:105F500007260AD077FD04D086D006D000201AF498
:105F6000709561957F4F0895F6F7909581959F4FB5
:105F70000895A1E21A2EAA1BBB1BFD010DC0AA1F8A
:105F8000BB1FEE1FFF1FA217B307E407F50720F0A2
:105F9000A21BB30BE40BF50B661F771F881F991F1D
:105FA0001A9469F760957095809590959B01AC0166
:105FB000BD01CF01089597FB092E05260ED057FD90
:105FC00004D0D7DF0AD0001C38F4509540953095A6
:105FD00021953F4F4F4F5F4F0895F6F7909580956D
:105FE000709561957F4F8F4F9F4F08952F923F92ED
:105FF0004F925F926F927F928F929F92AF92BF92D9
:10600000CF92DF92EF92FF920F931F93CF93DF9384
:10601000CDB7DEB7CA1BDB0B0FB6F894DEBF0FBEE1
:10602000CDBF09942A88398848885F846E847D842E
:106030008C849B84AA84B984C884DF80EE80FD8030
:106040000C811B81AA81B981CE0FD11D0FB6F894A6
:10605000DEBF0FBECDBFED010895EE0FFF1F05900F
:10606000F491E02D0994AA1BBB1B51E107C0AA1FA4
:10607000BB1FA617B70710F0A61BB70B881F991FE9
:106080005A95A9F780959095BC01CD01089591117D
:1060900006C0803219F089508550D0F708959927AD
:0860A00088270895F894FFCF52
:1060A8004E6F005965730054582074696D656F759B
:1060B8007421006D6F64756C65206C6F636B65642B
:1060C8003F00486F70206368616E6E656C20002029
:1060D80040200053004E2F4100386368002C002CEC
:1060E800205B005D20280029004E4F5420454E417A
:1060F800424C45440053656E64696E67207365744D
:1061080074696E677320746F2052580A0052657361
:10611800657474696E672073657474696E6773203B
:106128006F6E2052580A0041626F72746564206570
:10613800646974730A00696E76616C6964207365BA
:106148006C656374696F6E000D0A496E76616C69DF
:106158006420696E707574202D20646973636172A0
:106168006465642107007363616E6E6572206D6FEC
:1061780064650053657474696E677320736176652E
:106188006420746F20454550524F4D0A0052657681
:1061980065727465642073657474696E67732066CC
:1061A800726F6D20454550524F4D0A004C6F616427
:1061B800656420666163746F7279206465666175D1
:1061C8006C74730A004B657920616E6420636861A2
:1061D8006E6E656C732072616E646F6D697A65644A
:1061E8000A004F70656E4C52536E672054582073E6
:1061F80074617274696E672000206F6E20485720A2
:106208000050504D005253534900534441005343EA
:106218004C00525844005458440041494E004C42E6
:106228004545500053504B54524D0053425553006E
:1062380053554D44004C4C494E440000342B340017
:106248003800382B340031320031322B34003136EB
:106258000001000000C01200001A400AA1204EA54B
:10626800001B1E27522C23308025000005400AA160
:10627800204EA50020244EA52C2330004B000006FC
:10628800400AD0009D49007B289D492C233000E11D
:10629800000005400A4501D7DC03B81E0EBF0023E5
:1062A8002E48E801008A400A6001555502AD1E20BB
:1062B800000023C88025000005400AA1204EA50043
:1062C80020244EA52C233000020002000200020008
:1062D80002000200020002000200020002000200A6
:1062E80002000200020002FF01610265026A026EFA
:1062F80002720276027A027E0284028B0290029572
:10630800029B029B029B029B0235019C02A002A2F7
:1063180002A602A902AE02350100070B0C101115E6
:1063280000160A1322312900000000F32E622B8088
:086338002EBA2E9A2EE32E006E
:107E00000F92CDB7DEB7112484B714BE81FFF1D035
:107E100082E08093C00088E18093C10086E0809377
:107E2000C20080E18093C4008EE0CDD088249924E4
:107E3000CC24C394F5E0DF2EE1E1EE2E73E0F72EC3
:107E4000B6D0082F813479F4B2D08983C2D0898129
:107E5000823811F481E005C0813811F485E001C059
:107E600083E09ED09AC0823411F484E103C085344B
:107E700019F485E0B6D091C0853561F498D0082F0B
:107E800010E095D090E0982E8824802A912A880CC2
:107E9000991C82C0863521F484E0A3D080E0E1CF34
:107EA000843609F04CC083D082D0A82E80D0B82E62
:107EB00000E011E07CD0F80181938F01AE16D1F77C
:107EC00088D0FB2DF53489F4E0E0F1E00BC0F9999E
:107ED000FECF92BC81BC0894811C911C819180BD15
:107EE000FA9AF99AEA1598F358C08B2D863409F05E
:107EF00054C0F401F7BEE89507B600FCFDCFF401CD
:107F0000A0E0B1E02C9130E011968C91119790E0B7
:107F1000982F8827822B932B12960C01C7BEE895C9
:107F20001124329681E0A038B80761F7F401D7BE7A
:107F3000E89507B600FCFDCFE7BEE8952EC0843774
:107F4000F1F435D034D0182F32D0B82E42D0FB2DDA
:107F5000F63421F4F40105914F010CC0FB2DF534EA
:107F600049F4F999FECF92BC81BC0894811C911C04
:107F7000F89A00B5802F14D0115049F70EC08537FC
:107F800039F427D08EE10CD085E90AD08FE069CF93
:107F9000813511F488E017D01CD080E101D050CF9A
:107FA0009091C00095FFFCCF8093C600089580910A
:107FB000C00087FFFCCF8091C00084FD01C0A89560
:107FC0008091C6000895E0E6F0E098E19083808318
:107FD0000895EDDF803219F088E0F5DFFFCF84E10E
:107FE000DFCF1F93182FE3DF1150E9F7F2DF1F9166
:0E7FF0000895282E80E0E7DFEE27FF27099492
:027FFE0001057B
:0400000300007E007B
:00000001FF
